:100000000C945B000C94D9010C9406020C948300B0
:100010000C9483000C9483000C9483000C94830054
:100020000C9483000C9483000C9483000C94830044
:100030000C9483000C9483000C9483000C94830034
:100040000C9433020C9483000C9478030C9483007A
:100050000C9483000C9483000C9483000C94830014
:100060000C9483000C948300000024272A000025B0
:10007000282B000023262904040404040404040299
:100080000202020202030303030303010204081035
:100090002040800102040810200102040810200002
:1000A0000000070002010000030406000000000039
:1000B00000000000CE0111241FBECFEFD4E0DEBF50
:1000C000CDBF11E0A0E0B1E0E8ECF7E002C00590A0
:1000D0000D92A831B107D9F711E0A8E1B1E001C054
:1000E0001D92AE3AB107E1F710E0C6EBD0E004C0D4
:1000F0002297FE010E94DE03C43BD107C9F70E948C
:10010000C7010C94E2030C94000061E080910001AF
:100110000E94250360E0809102010E94250360E0B7
:10012000809104010E94250360E0809106010E94F5
:1001300025036091100170911101882777FD80954A
:10014000982F0E94A30261E0809100010E94250384
:1001500061E0809102010E94250360E0809104012A
:100160000E94250360E0809106010E9425036091B2
:10017000100170911101882777FD8095982F0E94BA
:10018000A30261E0809100010E94250361E080915B
:1001900002010E94250361E0809104010E94250371
:1001A00060E0809106010E9425036091100170912A
:1001B0001101882777FD8095982F0E94A30261E0A6
:1001C000809100010E94250361E0809102010E945C
:1001D000250361E0809104010E94250361E0809184
:1001E00006010E942503609110017091110188277A
:1001F00077FD8095982F0E94A30261E08091000115
:100200000E94250361E0809102010E94250361E0C4
:10021000809104010E94250360E0809106010E9404
:1002200025036091100170911101882777FD809559
:10023000982F0E94A30261E0809100010E94250393
:1002400061E0809102010E94250360E08091040139
:100250000E94250360E0809106010E9425036091C1
:10026000100170911101882777FD8095982F0E94C9
:10027000A30261E0809100010E94250360E080916B
:1002800002010E94250360E0809104010E94250381
:1002900060E0809106010E94250360911001709139
:1002A0001101882777FD8095982F0E94A30260E0B6
:1002B000809100010E94250360E0809102010E946C
:1002C000250360E0809104010E94250360E0809195
:1002D00006010E9425036091100170911101882789
:1002E00077FD8095982F0E94A302089561E0809188
:1002F00000010E94070361E0809102010E94070350
:1003000061E0809104010E94070361E08091060191
:100310000E94070361E0809108010E94070361E0E9
:1003200080910A010E94070361E080910C010E9404
:10033000070361E080910E010E94070360E0809155
:1003400000010E94250360E0809102010E942503C4
:1003500060E0809104010E94250360E08091060125
:100360000E94250361E0809108010E94250361E05D
:1003700080910A010E94250361E080910C010E9496
:10038000250361E080910E010E94250308950E94DB
:10039000CD020E9476010E948500FDCF86E191E0AA
:1003A00090931901809318010895862F0E9470037D
:1003B00008951F920F920FB60F9211242F933F931F
:1003C0004F935F936F937F938F939F93AF93BF935D
:1003D000EF93FF9380911A0190911B01892B29F0D3
:1003E000E0911A01F0911B010995FF91EF91BF91E6
:1003F000AF919F918F917F916F915F914F913F91BD
:100400002F910F900FBE0F901F9018951F920F9273
:100410000FB60F9211242F933F934F935F936F93D7
:100420007F938F939F93AF93BF93EF93FF938091AD
:100430001C0190911D01892B29F0E0911C01F09184
:100440001D010995FF91EF91BF91AF919F918F9100
:100450007F916F915F914F913F912F910F900FBEC0
:100460000F901F9018951F920F920FB60F921124A4
:100470002F938F939F93AF93BF9380911E01909181
:100480001F01A0912001B09121010196A11DB11D74
:1004900080931E0190931F01A0932001B09321012E
:1004A0008091220190912301A0912401B091250116
:1004B0008050904CAF4FBF4F809322019093230107
:1004C000A0932401B093250127C08091220190912F
:1004D0002301A0912401B091250180589E43A040A2
:1004E000B0408093220190932301A0932401B09304
:1004F00025018091260190912701A0912801B091BA
:1005000029010196A11DB11D809326019093270119
:10051000A0932801B0932901809122019091230199
:10052000A0912401B091250181589E43A040B04084
:1005300060F6BF91AF919F918F912F910F900FBE59
:100540000F901F901895EF92FF920F931F937B01CE
:100550008C018FB7F894409126015091270160914A
:100560002801709129018FBF2FB7F894809126013F
:1005700090912701A0912801B09129012FBF841BE0
:10058000950BA60BB70BE816F9060A071B0760F7D1
:100590001F910F91FF90EF900895789484B5826039
:1005A00084BD84B5816084BD85B5826085BD85B517
:1005B000816085BDEEE6F0E0808181608083E1E8C6
:1005C000F0E0808182608083808181608083E0E8C8
:1005D000F0E0808181608083E1EBF0E080818460E5
:1005E0008083E0EBF0E0808181608083EAE7F0E0E7
:1005F000808184608083808182608083808181604B
:1006000080838081806880831092C1000895282FA4
:1006100030E0C90185579F4FFC01949129583F4F05
:10062000F9018491882381F0E82FF0E0E859FF4F29
:10063000E491F0E0662329F48081909589238083FA
:1006400008958081892B80830895482F50E0CA0146
:1006500081569F4FFC012491CA0185579F4FFC0191
:10066000949149585F4FFA0134913323C1F1222309
:1006700031F1233021F4809180008F7705C0243040
:1006800031F4809180008F7D8093800018C02130EC
:1006900019F484B58F7704C0223021F484B58F7D9E
:1006A00084BD0DC0263021F48091B0008F7705C045
:1006B000273029F48091B0008F7D8093B000E32F24
:1006C000F0E0E359FF4FE491F0E0662329F48081E4
:1006D00090958923808308958081892B8083089554
:1006E000982F8091C00085FFFCCF9093C60008959D
:1006F0001F920F920FB60F9211242F933F934F9397
:100700005F936F937F938F939F93AF93BF93EF9379
:10071000FF934091C600E0912A01F0912B01CF0197
:10072000019660E870E00E94B5039C0180912C0165
:1007300090912D012817390739F0E25DFE4F408373
:1007400030932B0120932A01FF91EF91BF91AF913C
:100750009F918F917F916F915F914F913F912F91D9
:100760000F900FBE0F901F90189597FB092E07262C
:100770000AD077FD04D00CD006D000201AF4709572
:1007800061957F4F0895F6F7909581959F4F089555
:10079000AA1BBB1B51E107C0AA1FBB1FA617B707A7
:1007A00010F0A61BB70B881F991F5A95A9F78095C3
:1007B0009095BC01CD010895EE0FFF1F0590F491B7
:0807C000E02D0994F894FFCF2D
:1007C80006000700080009000200030004000500F5
:0807D800640000000000D501DF
:00000001FF
